:020000040000FA
:06000000020091022CC178
:0300230002294E61
:03002B00022CD5CF
:10003B00022B9953D9BF79012200000080FB1200DB
:10004B003EB9000302008BE4901000785B790880C6
:10005B0002F0A3D8FCD9FA90175AAA82AB8390006E
:10006B00A0781A79028015E493A3AC82AD838A82BF
:10007B008B83F0A3AA82AB838C828D83D8E9D9E7DB
:10008B00122D5712004475D0007581BF7510007585
:10009B001110020049506C656173652070726573B5
:1000AB007320616E79206B657920746F20636F6E9E
:1000BB0074696E75652E2E2E203F007C205452499C
:1000CB0047207C203530306E732F64207C203235F6
:1000DB002E30562F64207C2032352E30562F642044
:1000EB007C3F007C2053796E63207C20496E74200A
:1000FB007C205A20434841207C205A2043484220F0
:10010B007C204143204143207C3F0032352E30562A
:10011B002F643F0041433F0050432052554E204D2A
:10012B004F44453F0044433F00496E743F005379B1
:10013B006E633F0072616E67653A00000259802062
:10014B0054524947203F000000203530306E732F4A
:10015B0064203F2032352E30562F64203F2032351D
:10016B002E30562F64203F2053796E63203F0000C2
:10017B000020496E74203F00000000205A204348A5
:10018B0041203F0000205A20434842203F000020DE
:10019B00464654203F000000000000000000000015
:1001AB0000000001E52FE6FF00F801400707CAC079
:1001BB00E0E6F0A308DAFAD0E0FA22C3E498F8E418
:1001CB0099F91202078026C3E49AFAE49BFBE92013
:1001DB00E7E9120207E498F8E499F922C3E498F8E6
:1001EB00E499F9120207E498F8E499F9C3E49AFA4E
:1001FB00E49BFB22EB20E7CFE920E7E0B90010BB43
:10020B000008E88AF084F8AAF022E4FBC8FA22EB93
:10021B0070227B10C833C8C933C9335007C39AC384
:10022B00DBF280069A50012ADBEAC833F4C8C933E3
:10023B00F4C9FA2275F008E4C833C8C933C933C905
:10024B009AC99B5004C92AC93BD5F0ECFBC833F4BF
:10025B00C8E4C9FA22600D08C6A2E713C618C61374
:10026B00C6D5E0F322700422600D18C6C333C6084E
:10027B00C633C6D5E0F41822251010AF08F5104090
:10028B000215118008F51040021511D2AF22C0D013
:10029B00251010AF08F510500205118008F510500D
:1002AB00020511D2AFD0D0222510F58210AF08F580
:1002BB0010400215118008F51040021511D2AF85C0
:1002CB001183222510F582E43511F583222510C503
:1002DB0082C0E0E51134FFC583C0E0E510C3958211
:1002EB0024F9F8E4C5A8858311858210C5A8E8CE4A
:1002FB00F0A3E520F0A37808E608F0A3DEFAEFF010
:10030B00A3E58124FBF8E608F0A3E608F0A30808B0
:10031B00E608F0A3E608F0A315811581D0E0FED026
:10032B00E0F815811581E8C0E0EEC0E0228511836D
:10033B00851082E0A3FEE0A3F5207808E0A3F60881
:10034B00DFFAE0A3FFE0A3C0E0E0A3C0E0E0A3C0BE
:10035B00E0E0A3C0E0E4C5A8858210858311C5A8A1
:10036B00D083D0822274028000C0E0F4041202B366
:10037B00D0E01201B922D083D082C5F0E493A3C59B
:10038B00F0C395F0F5F0E493A3C395F04005E5F0C9
:10039B00048001E475F002A42582F582E5F0358333
:1003AB00F583E493A3C0E0E493C0E022D083D08232
:1003BB00E9C0E0E493A3C386F0C5F095F0F908E437
:1003CB0093A386F0C5F095F0700BE493A3C399400B
:1003DB0005E9048002A3E475F002A42582F582E509
:1003EB00F03583F583D0E0F9E493A3C0E0E493C048
:1003FB00E022D083D082CCC0E0E493A36006120449
:10040B00271470FAE493A360061204461470FAD012
:10041B00E0FCE493A3C0E0E493C0E022C0E0E493EB
:10042B00A3D39C5010E493A3C39C400AD0E0D0E02C
:10043B00D0E002041AA3A3A3D0E022C0E0E493A36C
:10044B006C7009D0E0D0E0D0E002041AA3A3D0E096
:10045B0022008040C020A060E0109050D030B070DF
:10046B00F0088848C828A868E8189858D838B87889
:10047B00F8048444C424A464E4149454D434B474AD
:10048B00F40C8C4CCC2CAC6CEC1C9C5CDC3CBC7C29
:10049B00FC028242C222A262E2129252D232B272A7
:1004AB00F20A8A4ACA2AAA6AEA1A9A5ADA3ABA7A29
:1004BB00FA068646C626A666E6169656D636B6764D
:1004CB00F60E8E4ECE2EAE6EEE1E9E5EDE3EBE7EC9
:1004DB00FE018141C121A161E1119151D131B17174
:1004EB00F1098949C929A969E9199959D939B979F9
:1004FB00F9058545C525A565E5159555D535B5751D
:10050B00F50D8D4DCD2DAD6DED1D9D5DDD3DBD7D98
:10051B00FD038343C323A363E3139353D333B37316
:10052B00F30B8B4BCB2BAB6BEB1B9B5BDB3BBB7B98
:10053B00FB078747C727A767E7179757D737B777BC
:10054B00F70F8F4FCF2FAF6FEF1F9F5FDF3FBF7F38
:10055B00FF00402060105030700848286818583849
:10056B007804442464145434740C4C2C6C1C5C3C84
:10057B007C02422262125232720A4A2A6A1A5A3A8E
:10058B007A06462666165636760E4E2E6E1E5E3E44
:10059B007E0141216111513171094929691959397B
:1005AB007905452565155535750D4D2D6D1D5D3D34
:1005BB007D03432363135333730B4B2B6B1B5B3B3E
:1005CB007B07472767175737770F4F2F6F1F5F3FF4
:1005DB007F00402060105030700848286818583849
:1005EB007804442464145434740C4C2C6C1C5C3C04
:1005FB007C02422262125232720A4A2A6A1A5A3A0E
:10060B007A06462666165636760E4E2E6E1E5E3EC3
:10061B007E014121611151317109492969195939FA
:10062B007905452565155535750D4D2D6D1D5D3DB3
:10063B007D03432363135333730B4B2B6B1B5B3BBD
:10064B007B07472767175737770F4F2F6F1F5F3F73
:10065B007F00000000000000000000000000000010
:10066B0000000000000010000000000000001E0051
:10067B000000000000001FC00000000000001FF879
:10068B000000000000000FFF00000000000001FF51
:10069B00E00000000000003FFC000000000000072D
:1006AB00FC00000000000000FC0000000000000047
:1006BB00FC00000000000003F80000000000000731
:1006CB00E0000018E801000FC0000018EC00001F4C
:1006DB00800000181E00007E000000180E8000FC39
:1006EB000000001803C001F80000001801E107F03A
:1006FB000000001800790FC000000018003E1F809A
:10070B0000000018000E1FC00000001800031FF8A7
:10071B0000000018000F0FFF00000018000D01FF74
:10072B00E00000180079003FFC00001800F0000703
:10073B00FC00001801C00000FC0000180380000042
:10074B001C00001807018000000000181C000000AE
:10075B00000000181800000000000008B000100096
:10076B0000000009F0001E0000000019C0001FC0AF
:10077B000000001F01199FF80000001E99001FFFC9
:10078B00000098DC000019FFE00880380000183FDB
:10079B00E008007800011837E00001D8000118309C
:1007AB00E00001880000183060000B1800001830C2
:1007BB0060000E080000183060001C180000183094
:1007CB0060007808000198306000E01800001830D5
:1007DB006001C008000018006007800800001800C6
:1007EB00600F0018000008006012000800000000F5
:1007FB00601C0018000180006078000800000000F9
:10080B00607000180000000060600008000010001D
:10081B00003C000800001E00001F000800009FC0E5
:10082B000007800800019FF80001E80800000FFF97
:10083B0000007808000001FFE0002E080000003FD8
:10084B00E0000B8800008007E00001C808898000E9
:10085B00E000017C88880000000000FC880000009C
:10086B000000489E000010000008801F40001E0082
:10087B0000000009D0019FC000000008F4001FF821
:10088B000000000C2C001FFF000000080F8019FF58
:10089B00E00000080580183FE000000C00C01807BE
:1008AB00E000000800F99800E000000C003C180084
:1008BB0000000008000F18000000000C00071800D3
:1008CB0000000008000318000000000C0006980050
:1008DB000000000C001C98000000000800381800F5
:1008EB000000000C006808000000000800E0000099
:1008FB000000000C0380800000000008070080004F
:10090B000000000C1C000000000000081800000094
:10091B000000000838000E000000000CE0001F0073
:10092B0000400008C0009F800000000F84881F80DB
:10093B000000000EC8001D8F00000C5C00001C1F87
:10094B00E044845C00001C1FF804C07C00001C1FEA
:10095B00F800006C00009C1CFC0001AC00001C1C8F
:10096B001C00038C00001C1C1C00070C00001C1C32
:10097B001C401C0800001C1C1C00180400009C1CC4
:10098B001C00680400009C1C1C00E00C00001C1CDC
:10099B001C01800C00001C1C1C03800C00001E1C86
:1009AB001C46000400009FDC1C1A000C00008FFC8E
:1009BB001C180004000007FC1C380004000001FC9C
:1009CB007C70000C000000387C7B000400000000F1
:1009DB007C4F000C000080007C05A0040000000090
:1009EB000000E80C0000000000003E0400000000C6
:1009FB0000000F0C00000000004003A4001F9E002D
:100A0B00000002E42AFF9FC00000007C7FC01FF89B
:100A1B00000000FFC0001FFF0000BFAE800019FFE9
:100A2B00C07FD00DC000983FE0200005B80018072C
:100A3B00E00000041A001800E00000040E0018008B
:100A4B006000000407C018006000000401C018001B
:100A5B00604000040078980060000004001C18003F
:100A6B0060000004000718006000000400079E00EF
:100A7B006000000400019F806040000400038F8829
:100A8B0060400004000E878F60000004000801071F
:100A9B00E000000400380007E000000400F0000351
:100AAB00E000000402800000C04000040180000050
:100ABB0000000004060000000000000416001E00E9
:100ACB00000000041C001FC00000000448001FF8B9
:100ADB0000000004E0001FFF00400004C04419FFA9
:100AEB00C00000078400183FE000002E000018072C
:100AFB00E000040C00001800E000041C00001800CB
:100B0B006044003400001800600000500000180022
:100B1B00600000E40000180060000384000018006F
:100B2B00600005040000180060400C040000180071
:100B3B0060001804000018006000780400001E001C
:100B4B006000400400001FC06001C00400000FF8EB
:100B5B0060038000000007FF60450004000001FFF8
:100B6B00E00C00000000003FE0180004000000074C
:100B7B00E010000400000000C0180002000000009C
:100B8B00003E0004000000000005A004000000006F
:100B9B000000D000000010000000110400001E0037
:100BAB0000000E0000001FC0000005C000001FF871
:100BBB00000001E400000FFF00000034000001FF03
:100BCB00E000001E4000007FE0000047800000674F
:100BDB00E0002004E0000060E0400000AC0000609A
:100BEB00600000000E000060600000040320006045
:100BFB0060000004012000606000000401600060E0
:100C0B0060000000003C006060000000000E00600F
:100C1B0060000000000300606000000400018078A9
:100C2B00600000000001807FE00000000002003F38
:100C3B00E00000040006001FE0000000000C0007AD
:100C4B00E000000400180000C00000040060100069
:100C5B000000000400A01E000000000401801FC063
:100C6B000000000407801FF80000000004001FFFB5
:100C7B00000000000C0019FFE00000043800183FD2
:100C8B00E0000004A0001837E0000000E00018307E
:100C9B00E0000003800018306000000700001830EF
:100CAB0060000006000018306000000C00001830D7
:100CBB0060000018000018306000001400001830AD
:100CCB00600000E0000018006000018400001800C4
:100CDB006000040000000800600006040000000033
:100CEB006000120400000000600010000000000013
:100CFB0060002004000000006000600000000000A5
:100D0B000000C00000000000000180040000000093
:100D1B000002000000000000000C000000000000BA
:100D2B000008000400000000000C0004000000009C
:100D3B0000058004000000000001400400000000DA
:100D4B00000030000000000000001D040000000047
:100D5B0000000D4000000000000000D0000000006B
:100D6B00000000B0000000000000001400000000B4
:100D7B000000000000000000000000000000100058
:100D8B000000000000001C000000000000001E001E
:100D9B000000000000001F000000000000001F000A
:100DAB000000000000001F810000000000001F81F8
:100DBB00E000000000001DC1F800000000001DC194
:100DCB00F800000000001CE0FC003FF01FF81CE0E6
:100DDB001C003FF01FF81C701C00030001981C70D6
:100DEB001C00030001981C381C00030001981C38E0
:100DFB001C00030001981C1C1C00030001981C1C08
:100E0B001C00030000181E0E1C00030000181FC658
:100E1B001C00030000180FC71C003FF0000007C3A5
:100E2B00FC003FF000000183FC0000000008000103
:100E3B00FC00000000780000FC00000001F0000046
:100E4B00080000000F800000000000101E000000D2
:100E5B00000000F01E000000000003E0078000000F
:100E6B0000001F0000F0100000003C0000381E00C6
:100E7B0000003C0000F81E0000000F0003C01E0025
:100E8B00000001E01E001E00000000701C000E00A0
:100E9B00000001F00F0000000000078001E00000DF
:100EAB0000003C0000780000000038000008000043
:100EBB0000001E0000000000000003C00000000046
:100ECB00000000F000000000000000100000000017
:100EDB0000000000000000000000000000000E00F9
:100EEB000000000000001FC00000000000001FF801
:100EFB000000000000001FFF0000000000001DFFAD
:100F0B00E000000000041C3FF800000000041C0778
:100F1B00F800000000061C00FC0000001FFE1C0077
:100F2B001C0000001FFE1C001C00000000001C0029
:100F3B001C001C3800001C001C003C3C00001C006A
:100F4B001C00300C00001C001C00300C00001C00AE
:100F5B001C00300C00001C001C00318C00001C001D
:100F6B001C00318C00001E001C00318C00001FC0C7
:100F7B001C00318C00000FF81C00318C000007FFA7
:100F8B001C003FFC000001FFFC001F780000003F2D
:100F9B00FC00000000000007FC0000000000000047
:100FAB00FC0000001C000000000000001C00000002
:100FBB00000000001C00000000000000000000000A
:100FCB0000003800000000000000380000000000A6
:100FDB0000003800000000000000000000000000CE
:100FEB000000000000000000000000000E1C0000CC
:100FFB00000000001E1E000000000000180600008C
:10100B000000000018060000000019F01806000090
:10101B00000030FC18C60000000030CC18C60000E1
:10102B00000030CC18C60000000030CC18C6000001
:10103B00000030CC18C60000000030CC1FFE0000B2
:10104B00000030CC0FBC0000000030CC00000000D2
:10105B00000030CC000000000000198C00000000E4
:10106B0000001F800000000000000F0000000000C7
:10107B000000000000000000000000001FFE000048
:10108B00000000001FFE000000000000180600001A
:10109B000000000018060000000000001806000009
:1010AB0000000000180600000000000018060000F9
:1010BB0000000000180600000000000018060000E9
:1010CB000000000018060000000000001C0E0000CD
:1010DB00000000000E1C00000000000007F80000DC
:1010EB000000000003F00000000000000000000002
:1010FB0000000000000000000000000000000000E5
:10110B0000000000000000000000000000000000D4
:10111B0000000000000000FF33FF33000000000060
:10112B000000000700070000000000070007000098
:10113B00002001FE1FFE1F20012001FE1FFE1F20AD
:10114B000138063C0E6408FF3FFF3F84091C0F1853
:10115B00071E30331C1E07C00170001C1E07330115
:10116B001E1E1FB331E120E120B3311E1F001B8077
:10117B00310000000000000B000700000000000021
:10118B000000000000F807FF3F07380000000000D8
:10119B000000000000000000000000000000000044
:1011AB000000000000000000000000000000000034
:1011BB000000000000000000000000000000000024
:1011CB000000000000000000000000000000000014
:1011DB000000000000000000000000000000000004
:1011EB000000000000000000300030000000000094
:1011FB00000030003C000FC003F0003C000F000368
:10120B0000FC0FFE1F0336812161201B30FE1FFCEB
:10121B000F042004200620FF3FFF3F00200020008A
:10122B00200C380E3C032601238121C3207E203C59
:10123B0020061803304120412041204120E330BEDD
:10124B001F000FE00FFC081F08833F803F000800C2
:10125B00083F0C3F1C2130212021206130C11F8110
:10126B000FE00FF81F5C3046204320C130811F0177
:10127B000F010001000100013C813FF1037F000FD2
:10128B00001C0FBE1FE33041204120E330BE1F1C6A
:10129B000F3C207E20C32081308118830EFE07FC7B
:1012AB000100000000000000000000000000000032
:1012BB000000000000000000000000000000000023
:1012CB000000000000000000000000000000000013
:1012DB0000200120012001200120012001200120FC
:1012EB0001000000000000000000000000000000F2
:1012FB0000000000000000000000000000000000E3
:10130B0000000000000000000000000000000000D2
:10131B0000FC3FFE3F0301010101010301FE3FFC05
:10132B003FFF3FFF3F412041204120E330BE1F1CC8
:10133B000FFC0FFE1F03300120012003300E1C0C8D
:10134B000CFF3FFF3F0120012001200738FE1FF853
:10135B0007FF3FFF3F412041204120412041200119
:10136B0020FF3FFF3F810081008100810081000150
:10137B0000FC0FFE1F03300120812083308E1F8C59
:10138B000FFF3FFF3F4000400040004000FF3FFF8A
:10139B003F012001200120FF3FFF3F0120012001E1
:1013AB0020000C001C0030002000200030FF1FFF2D
:1013BB000FFF3FFF3FC000E00138071C0E0F3C033F
:1013CB0030FF3FFF3F0020002000200020002000C6
:1013DB0020FF3FFF3F7800C003C0037800FF3FFFB3
:1013EB003FFF3FFF3F1C007000C0010007FF3FFFA6
:1013FB003FF03FF87F0CC0048004800CC0F87FF0F6
:10140B003FFF3FFF3F810081008100C3007E003C16
:10141B0000000000000000000000000000000000C1
:10142B0000FF3FFF3F810081008101C31F7E3E3CD7
:10143B00203C0C7E1C6330E120C12183318E1F0CBC
:10144B000F030003000300FF3FFF3F0300030003F4
:10145B0000FF0FFF1F0030002000200030FF1FFF98
:10146B000F3F00FF01C00F003C003CC00FFF013FCE
:10147B0000FF01FF3F003EC001C001003EFF3FFFE8
:10148B000100000000000000000000000000000050
:10149B000000000000000000000000000000000041
:1014AB00000138013E8127C121612039201F20070F
:1014BB002000000000000000000000000000000001
:1014CB000000000000000000000000000000000011
:1014DB000000000000000000000000000000000001
:1014EB0000000000000000000000000000000000F1
:1014FB0000000000000000000000000000000000E1
:10150B0000000000000000000000000000000000D0
:10151B0000001E403F2021202120212011E03FC050
:10152B003FFF3FFF3F4010202020206030C01F8036
:10153B000F800FC01F603020202020202060304003
:10154B0010800FC01F6030202020204010FF3FFF75
:10155B003F800FC01F6032202220226022C03380C8
:10156B001320002000FE3FFF3F210021002300023B
:10157B00008007C00F6018201020104008E03FE0EB
:10158B003F00000000000000000000000000000011
:10159B0000000020202020E33FE33F00200020003C
:1015AB000000000000000000000000000000000030
:1015BB0000FC3FFC3F00060007800DC01860302088
:1015CB0020000001200120FF3FFF3F0020002000F2
:1015DB0000E03FE03F6000C01FC01F6000E03FC065
:1015EB003FE03FE03F4000200020006000C03F8014
:1015FB003F800FC01F6030202020206030C01F8034
:10160B000FE03FE03F400420082008600CC007803B
:10161B0003000000000000000000000000000000BC
:10162B0000E03FE03FC00040006000600060004011
:10163B0000C010E0312021202320262024603C40D4
:10164B0018000020002000FE1FFE3F20202020005D
:10165B0000E01FE03F0020002000200010E03FE0F2
:10166B003FF003F007001C00300030001CF007F0C7
:10167B00030000000000000000000000000000005C
:10168B00000000000000000000000000000000004F
:10169B0000E001E027002600380018000EE007E00C
:1016AB000120302038202C20262023A021E0206090
:1016BB0020000000000000000000000000000000FF
:1016CB0000000000000000FF3FFF3F000000000093
:1016DB0000000000000000000000000000000000FF
:1016EB0000000000000000000000000000000000EF
:1016FB0000000000000000000000000000000000DF
:10170B0000000000000000000000000000000000CE
:10171B0000000000000000000000000000000000BE
:10172B0000000102030405060708090A0B0C0D0E45
:10173B000F101112131415161718191A1B1C1D1E36
:10174B001F202122232425262728292A2B2C2D2E26
:10175B002F303132333435363738393A3B3C3D3E16
:10176B003F404142434445464748494A4B4C4D4E06
:10177B004F505152535455565758595A5B5C5D5EF6
:10178B005F000000000000000000000000000000EF
:10179B00000000000000000000000000000000003E
:1017AB00000000000000000000000000000000002E
:1017BB00000000000000000000000000000000001E
:1017CB00000000000000000000000000000000000E
:1017DB0000000000000000000000000000000000FE
:1017EB0000000000000000000000000000000000EE
:1017FB0000000000000000000000000000000000DE
:10180B00000C000B000A00090008000A0009000880
:10181B00003132356D3F3235306D3F3632356D3FED
:10182B00312E32353F322E35303F362E32353F3169
:10183B00322E353F32352E303FFFFF0000020004C1
:10184B00000600080012001C0026004E0062007605
:10185B00008A009E00B200C600EE0016012A013E6F
:10186B000166018E0156021E03E603020004000806
:10187B00003530306E733F312E3075733F322E3062
:10188B0075733F332E3075733F342E3075733F3580
:10189B002E3075733F31302075733F3135207573A2
:1018AB003F32302075733F34302075733F35302015
:1018BB0075733F36302075733F37302075733F3863
:1018CB00302075733F39302075733F31303075736D
:1018DB003F31323075733F31343075733F313530B2
:1018EB0075733F31363075733F31383075733F3216
:1018FB00303075733F33303075733F343030757320
:10190B003F35303075733F312E306D733F322E3093
:10191B006D733F342E306D733F3235306E733F3500
:10192B0030306E733F312E3075733F312E357573FA
:10193B003F322E3075733F322E3575733F35202075
:10194B0075733F372E3575733F31302075733F32CA
:10195B00302075733F32352075733F3330207573EC
:10196B003F33352075733F34302075733F3435204A
:10197B0075733F35302075733F36302075733F37A5
:10198B00302075733F37352075733F3830207573B2
:10199B003F39302075733F31303075733F313530FF
:1019AB0075733F32303075733F32353075733F3559
:1019BB00303075733F312E306D733F322E306D7377
:1019CB003F75B9807A14001AEA70FB43B9C0E5B9C8
:1019DB00E5B9A2E550FA75A90275B28322C082C09F
:1019EB00831219CC75A40D75A5E775A70175D40FD6
:1019FB0075D50775DF0175E10575E242D28875E48F
:101A0B0001D2A8C2AA75C80475CA0175CB01C2ADB3
:101A1B00759810538EF4E58E438E08858D8B758DDE
:101A2B00F353890FE589438920D28E74019018688E
:101A3B00F0D2BCD2ACD28C438922E589438E0CE523
:101A4B008E758CB075C18043E60175D80053D9BF34
:101A5B0075D90275DA4275DB4275FC0775EA07D258
:101A6B00DEC283D282D280C292D291D290D2B0C245
:101A7B0096D296D2AF022949D296D282D29275A62D
:101A8B00FFD291C291D291D283C29275A083C280B0
:101A9B00D280D29275A002C280D280C283D283C27E
:101AAB009275A085C280D280D29275A003C280D2DB
:101ABB0080C283D283C29275A08CC280D280D29214
:101ACB0075A093C280D280C283D283C29275A0913B
:101ADB00C280D280D29275A001C280D280C283D242
:101AEB0083C29275A083C280D280D29275A000C2AD
:101AFB0080D280C283D283C29275A03EC280D28034
:101B0B00D29275A0B0C280D280C283D283C29275AA
:101B1B00A03FC280D280D29275A003C280D280C275
:101B2B0083D283C29275A040C280D280D29275A01C
:101B3B0010C280D280C283D283C29275A041C28070
:101B4B00D280D29275A056C280D280C283D283C279
:101B5B009275A042C280D280D29275A013C280D25D
:101B6B0080C283D283C29275A043C280D280D292AC
:101B7B0075A046C280D280C283D283C29275A04424
:101B8B00C280D280D29275A023C280D280C283D26F
:101B9B0083C29275A045C280D280D29275A076C2C4
:101BAB0080D280C283D283C29275A046C280D2807B
:101BBB00D29275A000C280D280C283D283C29275AA
:101BCB00A047C280D280D29275A05EC280D280C262
:101BDB0083D283C29275A048C280D280D29275A064
:101BEB004FC280D280C283D283C29275A049C28079
:101BFB00D280D29275A040C280D280C283D283C2DF
:101C0B009275A017C280D280D29275A061C280D289
:101C1B0080C283D283C29275A02BC280D280D29213
:101C2B0075A0F9C280D280C283D283C29275A01BE9
:101C3B00C280D280D29275A014C280D280C283D2CD
:101C4B0083C29275A01AC280D280D29275A011C2A3
:101C5B0080D280C283D283C29275A01CC280D280F4
:101C6B00D29275A00DC280D280C283D283C29275EC
:101C7B00A01FC280D280D29275A03DC280D280C2FA
:101C8B0083D283C29275A019C280D280D29275A0E2
:101C9B000AC280D280C283D283C29275A019C2803D
:101CAB00D280D29275A01AC280D280C283D283C254
:101CBB009275A019C280D280D29275A012C280D226
:101CCB0080C283D283C29275A01EC280D280D29270
:101CDB0075A020C280D280C283D283C29275A03CF1
:101CEB00C280D280D29275A060C280D280C283D2D1
:101CFB0083C29275A03DC280D280D29275A040C2A1
:101D0B0080D280C283D283C29275A034C280D2802B
:101D1B00D29275A038C280D280C283D283C2927510
:101D2B00A035C280D280D29275A038C280D280C238
:101D3B0083D283C29275A024C280D280D29275A026
:101D4B0038C280D280C283D283C29275A024C28053
:101D5B00D280D29275A03CC280D280C283D283C281
:101D6B009275A016C280D280D29275A01CC280D26E
:101D7B0080C283D283C29275A001C280D280D292DC
:101D8B0075A006C280D280C283D283C29275A05541
:101D9B00C280D280D29275A000C280D280C283D280
:101DAB0083C29275A002C280D280D29275A000C26B
:101DBB0080D280C283D283C29275A003C280D280AC
:101DCB00D29275A000C280D280C283D283C2927598
:101DDB00A004C280D280D29275A000C280D280C2F1
:101DEB0083D283C29275A005C280D280D29275A095
:101DFB00EFC280D280C283D283C29275A006C2800A
:101E0B00D280D29275A000C280D280C283D283C20C
:101E1B009275A007C280D280D29275A000C280D2E8
:101E2B0080C283D283C29275A008C280D280D29224
:101E3B0075A001C280D280C283D283C29275A009E1
:101E4B00C280D280D29275A08FC280D280C283D240
:101E5B0083C29275A022C280D280D292C28375A611
:101E6B000075A0FF2275A6FFD283C29275A003C294
:101E7B0080D280D29289A0C280D280C283D283C208
:101E8B009275A006C280D280D292EBF5A0C280D20E
:101E9B0080C283D283C29275A007C280D280D292B5
:101EAB00EAF5A0C280D280C283D283C29275A022EF
:101EBB00C280D280D292C2832274F81202D87408E4
:101ECB001202CEE0FEA3E0FFD283C29275A002C243
:101EDB0080D280D29275A000C280D280C283D2837E
:101EEB00C29275A003C280D280D29289A0C280D246
:101EFB0080C283D283C29275A004C280D280D29258
:101F0B0075A000C280D280C283D283C29275A00515
:101F1B00C280D280D2928CA0C280D280C283D28364
:101F2B00C29275A006C280D280D292EBF5A0C2807D
:101F3B00D280C283D283C29275A007C280D280D2D4
:101F4B0092EAF5A0C280D280C283D283C29275A0DE
:101F5B0008C280D280D292EFF5A0C280D280C28319
:101F6B00D283C29275A009C280D280D292EEF5A024
:101F7B00C280D280C283D283C29275A022C280D289
:101F8B0080D292C28302237374F71202D87409129F
:101F9B0002CEE0F508A3E0F5097E987F9E75A6FFBB
:101FAB007808120370121EC47402120299D283C2F3
:101FBB009275A022C280D280D292C28390174EE03B
:101FCB00FAA3E0D283F5A0C280D280EAF5A0C2804A
:101FDB00D280C28390174EE0FAA3E0D283F5A0C261
:101FEB0080D280EAF5A0C280D280C283EEF8EFF9EE
:101FFB0074FF281E74FF39FFE87001E970BE750885
:10200B008F75090178081203707CEF7A007B0079D9
:10201B0000121EC4740212029902490174F81202D2
:10202B00D8EAFEEBFFD29675A6FF7A007B0079000B
:10203B00121E70D283C29275A022C280D280D2921D
:10204B00C2837AF97BC0EFFCD2838CA0C280D28092
:10205B00EEF5A0C280D280C283D2838CA0C280D284
:10206B0080F5A0C280D280C283EA1A70DBEB1B70B2
:10207B00D702237374F41202D8890BEC240CF5826B
:10208B00E43417F583E49390174BF0F508750900CA
:10209B0074037808120270901749E508F0A3E5095C
:1020AB00F08A088B09901749E0F8A3E0F9E8C333ED
:1020BB00F8E933F9E8240CFEE93411FF750A08AA94
:1020CB0008AB09A90B121E7078007920D283C2923B
:1020DB0075A022C280D280D292C283750C0E8E82E2
:1020EB008F83E49358FAA3E49359FBEA7001EB60F6
:1020FB000590174C800390174EE0FCA3E0D283F5BC
:10210B00A0C280D280ECF5A0C280D280C283E9C38A
:10211B0013F9E813F8150CE50C70C3EE24020E0E40
:10212B00EF3400FFE5082401F508E5093400F50953
:10213B00150AE50A708902342A74F11202D8890A49
:10214B00ECFEED8A0C8B0D75085C750906750E5649
:10215B00750F01F50BAA0CAB0DA90A121E70D283D9
:10216B00C29275A022C280D280D292C2838508828D
:10217B008509837B087C807A08E4935CD283600CAE
:10218B00850BA0C280D280EEF5A0800A75A074C228
:10219B0080D28075A053C280D280C283ECC313FC63
:1021AB001AEA70D5A31BEB70CCE5082408F508E5FB
:1021BB00093400F509E50C2401F50CE50D3400F5A7
:1021CB000DE50E24FFF50EE50F34FFF50FE50E7050
:1021DB0002E50F70808004C296D2967F0802033806
:1021EB0074F81202D890174EE4F0A3F090175074C5
:1021FB00BFF0A3741DF090174C74FFF0A3F0901771
:10220B004EE0FAA3E0FB122027901745E0D2E0F056
:10221B007C8F7D017A017B0079121223787C8F7D74
:10222B00017A017B0079011223787C8F7D017A0181
:10223B007B0079DF1223787C8F7D017A017B00791B
:10224B00EF1223787E007F007582807583178019CB
:10225B00EEFAEFFBEA75F00AA4FAADF075F00AEBB3
:10226B00A42DFB790212207FA3E0FAEE24010EEFDE
:10227B003400FFEAFC743F6A70D67E007F007582E3
:10228B00A87583178019EEFAEFFBEA75F00AA4FA2A
:10229B00ADF075F00AEBA42DFB79E112207FA3E0E2
:1022AB00FAEE24010EEF3400FFEAFC743F6A70D69D
:1022BB00901869E0F8A3E0F990174CE8F0A3E9F067
:1022CB007582D07583177EC87F008012EEFAEFFB04
:1022DB00790212207FEE240AFEEF3400FFA3E0FA0E
:1022EB00FC743F6A70E67582D97583177E407F0157
:1022FB008012EEFAEFFB79E112207FEE240AFEEF5B
:10230B003400FFA3E0FAFC743F6A70E690186BE0B0
:10231B00F8A3E0F990174CE8F0A3E9F07582D975B2
:10232B0083177E5E7F018012EEFAEFFB79E11220BC
:10233B007FEE240AFEEF3400FFA3E0FAFC743F6A41
:10234B0070E67582D07583177E2C7F018012EEFAB2
:10235B00EFFB790212207FEE240AFEEF3400FFA37D
:10236B00E0FAFC743F6A70E67F0102033874F612E0
:10237B0002D8890A8A088B09ECFEEDFF121E7090B9
:10238B001745E0A2E0E492E0120381000109249ECC
:10239B0023CA23901750E0FAA3E0D283F5A0C280A2
:1023AB00D280EAF5A0C280D280C283EEF8EFF97436
:1023BB00FF281E74FF39FFE87001E970D6803F904B
:1023CB001750E0FAA3E0D283F5A0C280D280EAF5E1
:1023DB00A0C280D280C283AA08AB09A90A121E70C0
:1023EB00E5082401F508E5093400F509EEF8EFF9E5
:1023FB0074FF281E74FF39FFE87001E970C17F0379
:10240B0002033874F71202D890175074EFF0A374CC
:10241B007BF07508197509007E147F00AA08AB09BB
:10242B00EEF9121E70901750E0FAA3E0D283F5A0DC
:10243B00C280D280EAF5A0C280D280C283EE24058E
:10244B00FEEF3400FFC3EE94E0EF940040CEE508BE
:10245B002419F508E5093400F509C3E508948FE55F
:10246B0009940140B37508147509007E007F00EED6
:10247B00FAEFFBA908121E70901750E0FAA3E0D2F6
:10248B0083F5A0C280D280EAF5A0C280D280C2833D
:10249B00EE2405FEEF3400FFC3EE948FEF94014062
:1024AB00CEE5082419F508E5093400F509C3E5085C
:1024BB0094E0E509940040B3901745E0C2E0F07C4E
:1024CB00C87D007AC87B007914122378E0D2E0F043
:1024DB007C8F7D017A007B00797812237802490189
:1024EB0074F51202D8901750E0F50AA3E0F50B90A3
:1024FB001750E4F0A3F090174EF0A3F0901745E0BF
:10250B00C2E0F07E127F007508297C0D7D00EEFA8B
:10251B00EFFB79021223787C0D7D0074012EFAE417
:10252B003FFB7902122378EE240AFEEF3400FF15ED
:10253B0008E50870D5E0C2E0F07E127F007508292F
:10254B007C0D7D00EEFAEFFB79E11223787C0D7D9B
:10255B000074012EFAE43FFB79E1122378EE240A92
:10256B00FEEF3400FF1508E50870D5901869E0F808
:10257B00A3E0F990174CE8F0A3E9F07E007F00751B
:10258B0008BE8E098015AA08AB09790212207FE5D7
:10259B0008240AF508E5093400F509EE2418F5823C
:1025AB00EF3418F583E0FAEE24010EEF3400FFEA66
:1025BB00FC743F6A70D090186BE0F8A3E0F99017A9
:1025CB004CE8F0A3E9F07E007F0075082275090145
:1025DB008015AA08AB09790212207FE508240AF5B9
:1025EB0008E5093400F509EE2422F582EF3418F5DD
:1025FB0083E0FAEE24010EEF3400FFEAFC743F6A2D
:10260B0070D0901743E0A2E790174C500874E0F09D
:10261B00A37407800474FFF0A3F07E007F0075089D
:10262B005A8E098015AA08AB0979E112207FE508BB
:10263B00240AF508E5093400F509EE2436F582EF96
:10264B003418F583E0FAEE24010EEF3400FFEAFCB8
:10265B00743F6A70D0901000E07011901869E0F828
:10266B00A3E0F990174CE8F0A3E980106401700522
:10267B0090186B80E990174C74FFF0A3F07E007FED
:10268B00007508148E098015AA08AB0979E1122090
:10269B007FE508240AF508E5093400F509EE242C3A
:1026AB00F582EF3418F583E0FAEE24010EEF3400D7
:1026BB00FFEAFC743F6A70D090174C74FFF0A3F0E4
:1026CB007E007F007508148E098015AA08AB097966
:1026DB000212207FE508240AF508E5093400F50904
:1026EB00EE2404F582EF3418F583E0FAEE24010EA4
:1026FB00EF3400FFEAFC743F6A70D07E007F0075F8
:10270B00085A8E098015AA08AB09790212207FE5B9
:10271B0008240AF508E5093400F509EE240EF582C4
:10272B00EF3418F583E0FAEE24010EEF3400FFEAE4
:10273B00FC743F6A70D07E007F007508968E09800E
:10274B0015AA08AB0979E112207FE508240AF508E0
:10275B00E5093400F509EE2440F582EF3418F583D2
:10276B00E0FAEE24010EEF3400FFEAFC743F6A70CE
:10277B00D07E007F007508E68E098015AA08AB098C
:10278B0079E112207FE508240AF508E5093400F504
:10279B0009EE244AF582EF3418F583E0FAEE2401B2
:1027AB000EEF3400FFEAFC743F6A70D0901750E5CF
:1027BB000AF0A3E50BF07F04020338C082C08374D8
:1027CB0001901736F0901746E04412F07959122811
:1027DB00C2901802E0901722F0901736E090172362
:1027EB00F0901737E0901724F0901738E0901725EA
:1027FB00F07402901736F0901746E04412F07959B6
:10280B001228C2901736E0901726F0901737E090F9
:10281B001727F0901738E0901728F07408901736A8
:10282B00F0901746E04412F079591228C2901736EF
:10283B00E0901729F0901737E090172AF09017388F
:10284B00E090172BF0740E901736F0901746E0C2FD
:10285B00E1F0D2E4F079591228C2901736E09017C4
:10286B002CF0901737E090172DF07437901736F047
:10287B00901746E0C2E1F0D2E4F079591228C290E9
:10288B001736E090172EF0901737E090172FF07453
:10289B000D901736F0901746E0C2E1F0D2E4F079D4
:1028AB00591228C2901736E0901730F0901737E086
:1028BB00901731F0022949C082C0837A007B0090C7
:1028CB001746A2A8E092E3F0C2A8E9901802F09094
:1028DB001746E0D2E0F0A2E45007C2E4F0D2E28067
:1028EB0002C2E2F0D2C5E0A2E0501BEAF8EBF974A9
:1028FB0001280AE439FBC3E894E9E994FD40ECE0D4
:10290B00C2E0F0C340E5901748E0A2E25028E0A2F5
:10291B00E14023E4901737F0901738F074019017CB
:10292B0036F0901746E0C2E2F0D2C5A2E040FC9030
:10293B001748E0C2E2F0901746E0A2E392A8D083DA
:10294B00D08222C0E0C0D0E8C0E0E9C0E0C082C0C5
:10295B0083A2984003022B19901719E07007901768
:10296B001CE4F0A3F0C298E599901721F090171989
:10297B00E0C394114003022B84901721E0C0E09038
:10298B00171CE02409F8A3E03417F988828983D057
:10299B00E0F0901719E004F090171CE02401F0A36D
:1029AB00E03400F0901719E064106003022B849060
:1029BB001718E0640D6003022B00901743E0A2E5AB
:1029CB00500B901717E0640A700343EF10901743F6
:1029DB00C082901709E0A2E0758317D082E092E3E2
:1029EB00F0901743C08290170AE0A2E0758317D0CE
:1029FB0082E092E1F0901743C08290170BE0A2E0C7
:102A0B00758317D082E092E2F0901743E0A2E14089
:102A1B000DE0A2E2400890170CE090173DF09017E4
:102A2B000DE0901737F090170EE0901738F09017D5
:102A3B000FE0901736F0901710E0901802F09017F7
:102A4B0011E0901803F0901712E0901720F09017F8
:102A5B0043C082901713E0A2E0758317D082E092F7
:102A6B00E6F0901720E064017004C2B08002D2B08F
:102A7B00901709E0602A64027008901803E0F5FCD7
:102A8B00800BE064037006901803E0F5EAC29690A1
:102A9B00173BE4F0A3F0D296901743E0C2E080100E
:102AAB00901743E0A2E140F3E0A2E240EEE0D2E077
:102ABB00F0901736E064017008901746E0D2E18081
:102ACB0010E0640260F3E0640860EE901746E0C229
:102ADB00E1F0901716E0600F901743E0C2E0F09022
:102AEB001744E0D2E38006901744E0C2E3F0E49091
:102AFB001719022B83E4901719F0901743E0D2E0DB
:102B0B00F0E0C2E3F0E0C2E1F0E0C2E2806AA29939
:102B1B005067C299901800E07002A3E0604B9018C8
:102B2B0000E0F8A3E0F990171AE0687003A3E069DE
:102B3B00700790171EE4F0A3F090171EE02401F825
:102B4B00A3E03410F988828983E0901721F0F5997E
:102B5B0090171EE02401F0A3E03400F0901800E081
:102B6B0024FFF0A3E034FF800F90171AE0F8A3E0E6
:102B7B00F9901800E8F0A3E9F0D083D082D0E0F907
:102B8B00D0E0F88004D083D082D0D0D0E032C0E047
:102B9B00C0D0C082C083C0F0A2C25003022CBA7452
:102BAB00F055C01203FD0003807F2CC0DB2BE0BE71
:102BBB002BBA2C901802E0C333F5C253C2FE901708
:102BCB0046E0A2E4E492E045C2F5C2C2C5022CBACB
:102BDB00A2C14003022C6E901746E0A2E450030200
:102BEB002CBA901739E064017023901802E0645DF1
:102BFB00600AE064486005E064497042901746E063
:102C0B00C2E0F0E4901739F0D2C4022CBA90174608
:102C1B00E0A2E14008901739E0640260DF901739B9
:102C2B00E01203810003BA2C3B2C492C632C072C9C
:102C3B00901739E004F0901736E0F5C280719017C9
:102C4B0046E0A2E25007D2E4F0D2C5806290173979
:102C5B00E004F090173780E1901739E004F09017FB
:102C6B003880D6E4901739F0D2C4901802E0645D36
:102C7B00603D80D5901739E01203810101BA2C8E8B
:102C8B002CA62CE5C2901737F0901739E004F09082
:102C9B001746E0A2E1500AD2C18014E5C290173862
:102CAB00F0C2C1E4901739F0901746E0C2E0F0C2D1
:102CBB00C0D0F0022B90C0E0C0D0C082C083D290B5
:102CCB00901743E0D2E4F0022B90C0E0C0D0EAC0F2
:102CDB00E0C082C08390186FE0FA74012AF0EAC357
:102CEB009405405C75A60075A0FFC296C283901731
:102CFB0047A2A5E092E0F0A2A0E092E1F0A2A6E04C
:102D0B0092E2F0A2A7E092E3F0A2A2E092E4F0A29A
:102D1B00A1E092E5F0A2A3E092E6F0A2A4E092E794
:102D2B00F0E064FF6013901748E0A2E4400BE0D2A0
:102D3B00E3F0901743E0C2E3F0D296E490186FF003
:102D4B00C2CFD083D082D0E0FA022B94901743E00D
:102D5B00C2E5F0901748E0D2E4F074FF901747F00B
:102D6B007402901000F0901744E0D2E0F0E0D2E152
:102D7B00F0D2B01219E8E5EFA2E4901743E05063EC
:102D8B00C2E5F0121A8390174CE4F0A374F8F07AB2
:102D9B00007B00122027901745E0D2E0F07C8F7D5E
:102DAB00017A017B00794F1223787C8F7D017A01A8
:102DBB007B00799F1223787582DD7583177E9A7F4E
:102DCB00008012EEFAEFFB797012207FEE240AFEE0
:102DDB00EF3400FFA3E0FAFC743F6A70E6901743F0
:102DEB00022EE1D2E5F07418901737F0744090176B
:102DFB0038F07402901736F0901748E0D2E2F0905A
:102E0B001746E0C2E4F0D2E1F0901748E0C2E1F0DF
:102E1B0079591228C2E0D2E2F0E490173AF09017F9
:102E2B0046E054EDF090173AE0901736F0795D12CA
:102E3B0028C2901746E054EDF07408901736F079DD
:102E4B00481228C2901746E054EDF07408901736DC
:102E5B00F079491228C2121A8375A6FF7A537B7434
:102E6B0012202790174C7437F0A374FFF090174E75
:102E7B007453F0A37474F07C377DFF7A237B007955
:102E8B005A12214475825A7583177E1E7F00801259
:102E9B00EEFAEFFB791912207FEE240AFEEF3400D5
:102EAB00FFA3E0FAFC743F6A70E6D2AD901747E0DF
:102EBB0064FF60F8901748E0C2E4F0C2AD1221EB5A
:102ECB0012240E901743E0D2E3800EC296D29612D4
:102EDB0031BEE0C2E3F0E0D2E0F0901743E0A2E5B0
:102EEB00500302300875A60075A0FFE0A2E040FB7E
:102EFB00E0A2E340D6E0A2E1501F1227C6901800D3
:102F0B007414F0A3E4F090171A7414F0A3E4F0D245
:102F1B0099901743E0C2E180BCE0A2E2501D9017EC
:102F2B0046E0C2E4F0901802E0F91228C274019056
:102F3B001868F0901743E0C2E2809A901744E0A221
:102F4B00E35097901715E0FA704B901716E0FEC3FD
:102F5B00940590173AE04004C2E08002D2E0F09072
:102F6B001746E054EDF090173AE0901736F0795D84
:102F7B001228C2901746E054EDF0EEC333F8E43359
:102F8B00F9E8240CF582E93418F583E493901736AD
:102F9B00F07948804E74016A704C901716E0FEC3AE
:102FAB00940590173AE04004C2E18002D2E1F09020
:102FBB001746E054EDF090173AE0901736F0795D34
:102FCB001228C2901746E054EDF0EEC333F8E43309
:102FDB00F9E8240CF582E93418F583E4939017365D
:102FEB00F079491228C2901743E0D2E0F0901744D1
:102FFB00E0C2E3022EE41227C6E0C2E1F0901743D1
:10300B00E0A2E540030231BD800AE0A2E15005C217
:10301B00AD12383BD2AD901743E0A2E3E0502FA2A4
:10302B00E75007C2AD123CDB80EA901744E0FAE0B0
:10303B00FBEAA2E0500CEBA2E15007C2AD1239C083
:10304B0080D2E0A2E050C3C2AD1236B680C6A2E178
:10305B0040A4E0A2E25021901746E0C2E4F09018A1
:10306B0002E0F91228C27401901868F0901743E03F
:10307B00C2E2F0E0D2E38084901748E0A2E3400381
:10308B00023008901743E0C2E2F0901747E0A2E24B
:10309B00407F90173AE06410F0901746E054EDF043
:1030AB0090173AE0901736F0795D1228C2901869A4
:1030BB00E0F8A3E0F990174CE8F0A3E9F090173A89
:1030CB00E0A2E440267582D97583177E407F01E02C
:1030DB00FAFC743F6A603AEEFAEFFB79E112207F5B
:1030EB00EE240AFEEF3400FFA380E47582EA7583B9
:1030FB00177E407F018012EEFAEFFB79E112207F01
:10310B00EE240AFEEF3400FFA3E0FAFC743F6A7072
:10311B00E6901747E0A2E3407F90173AE06420F077
:10312B00901746E054EDF090173AE0901736F0798F
:10313B005D1228C290186BE0F8A3E0F990174CE8E9
:10314B00F0A3E9F090173AE0A2E540267582D97515
:10315B0083177E5E7F01E0FAFC743F6A603AEEFAF9
:10316B00EFFB79E112207FEE240AFEEF3400FFA380
:10317B0080E47582EA7583177E5E7F018012EEFA1A
:10318B00EFFB79E112207FEE240AFEEF3400FFA360
:10319B00E0FAFC743F6A70E6C2AD123E86901748A7
:1031AB00E0C2E3F0901743E0A2E2500302300802C2
:1031BB00307E22C082C083D2A8C290901743E0A277
:1031CB00E450F8E0C2E4F0C2A8D29090173DE06062
:1031DB00046402704B90173BE4F0A3F07801791074
:1031EB00D297C297E5A088828983F0D29790173B3C
:1031FB00E02401F0A3E03400F088828983A3A88245
:10320B00A98390173BC3E094FFA3E0940140D1D274
:10321B0097E4901001F090171AF0A37402F0D29972
:10322B00901720E064016005E0640270089017437A
:10323B00E0A2E650F890173DE064016005E06402FF
:10324B00704B90173BE4F0A3F078017910D295C244
:10325B0095E5A088828983F0D29590173BE02401F5
:10326B00F0A3E03400F088828983A3A882A983901D
:10327B00173BC3E094FFA3E0940140D1740190107D
:10328B0001F090171AE4F0A37402F0D299C296D20F
:10329B009602294974F41202D8750A00E490175269
:1032AB00F075A60075A0FF782179137A10C297E507
:1032BB00A0245CF582E43404F583E493888289834B
:1032CB00F0D297A3A882A9831AEA70E1750B08784C
:1032DB00297913C297E82408FAE93400FBE5A02406
:1032EB005CF582E43404F583E4938A828B83F0D219
:1032FB0097E50A704E88828983E0F582AE8290183A
:10330B0070E0FC74FC2CF50874FF3400F509C3E580
:10331B00089EE5099400A2D265D033502674042C84
:10332B00FCE43400FDEE9CE49DC365D03350148A5D
:10333B00828B83E0FAEEC39A5009E50B901752F09B
:10334B00750A01050B88828983A3A882A983E50BE3
:10335B00C3945C50030232DE02342A74F41202D896
:10336B00750A00E4901752F075A60075A0FF78154A
:10337B0079157A10C295E5A0245CF582E43404F546
:10338B0083E49388828983F0D295A3A882A9831AB8
:10339B00EA70E1750B08781D7915C295E82408FAD7
:1033AB00E93400FBE5A0245CF582E43404F583E406
:1033BB00938A828B83F0D295E50A704E888289833B
:1033CB00E0F582AE82901870E0FC74FC2CF508746A
:1033DB00FF3400F509C3E5089EE5099400A2D26508
:1033EB00D033502674042CFCE43400FDEE9CE49D99
:1033FB00C365D03350148A828B83E0FAEEC39A50A4
:10340B0009E50B901752F0750A01050B8882898329
:10341B00A3A882A983E50BC3945C50030233A57F59
:10342B000502033874F21202D8750B00E4901752A0
:10343B00F075A60075A0FF782179137A157B157CA2
:10344B0010C297E5A0245CF582E43405F583E49380
:10345B0088828983F0D297C295E5A0245CF582E43B
:10346B003405F583E4938A828B83F0D295A3AA82E9
:10347B00AB8388828983A3A882A9831CEC70C27555
:10348B000A087A297B137C1D7D15C297EA2408F85C
:10349B00EB3400F9E8FEE9FFE5A0245CF582E434A7
:1034AB0005F583E4938E828F83F0D297C295EC243B
:1034BB0008F8ED3400F9880C890DE5A0245CF58241
:1034CB00E43405F583E49388828983F0D295E50B88
:1034DB00600302358A901000E070568A828B83E07D
:1034EB00F50EF582858208901870E0F874FC28F5CB
:1034FB000C74FF3400F50DC3E50C9508E50D940035
:10350B00A2D265D0335078740428F8E43400F9E57E
:10351B000898E499C365D03350658E828F83E0FEA3
:10352B00E50EC39E5059E50A901752F0750B0180BA
:10353B004E6401704A8C828D83E0F50EF582AE826B
:10354B00901870E0F874FC28F50874FF3400F50946
:10355B00C3E5089EE5099400A2D265D033502074D0
:10356B000428F8E43400F9EE98E499C365D033509D
:10357B000E850C82850D83E0FEE50EC39E40A705EC
:10358B000A8C828D83A3AC82AD838A828B83A3AAA0
:10359B0082AB83E50AC3945C50030234957F070228
:1035AB00033874F41202D87E00E4901752F075A61B
:1035BB000075A0FF782179137A08C297E5A0245CE7
:1035CB00F582E43404F583E49388828983F0D297FF
:1035DB00C295E5A0245CF582E43404F583E493887A
:1035EB00828983A3F0D295E824020808E93400F914
:1035FB001AEA70C67F0878297913C297E82408FA6B
:10360B00E93400FBE5A0245CF582E43404F583E4A3
:10361B00938A828B83F0D297C295E5A0245CF582C6
:10362B00E43404F583E49388828983A3A3A3A3A33F
:10363B00A3A3A3A3F0D295EE705A901000E06402FE
:10364B00605288828983E0F50CF582858208901898
:10365B0070E0FC74FC2CF50A74FF3400F50BC3E529
:10366B000A9508E50B9400A2D265D033502674045A
:10367B002CFCE43400FDE5089CE49DC365D033507D
:10368B00138A828B83E0FAE50CC39A5007EF9017ED
:10369B0052F07E010F0FE824020808E93400F9EF1D
:1036AB00C3945B500302360502342A74F11202D81C
:1036BB00D2A8C290901743E0A2E450F8E0C2E4F025
:1036CB00C2A812329F901000E0640270087401903F
:1036DB001752F08009901752E070030238387E00C1
:1036EB007F00750E85750F13750801750910E024A1
:1036FB0021F50CE43413F50D75A60075A0FFC297E8
:10370B00E5A0245CF582E43404F583E493850E8212
:10371B00850F83F0D29775A6FF850882850983E014
:10372B00FC74786C600874C86E7001EF700B9017A6
:10373B005074EFF0A3747B8052EC75F00584E5F0C8
:10374B007011EEF8EFF97A197B00120207EA70019B
:10375B00EB60DB8C0A7405250AF8E43400F97A195E
:10376B007B001201FFEA7001EB7011EEF8EFF97AB2
:10377B00057B00120207EA7001EB60B290174EE076
:10378B00F8A3E0F9901750E8F0A3E9F0EEFAEFFB9D
:10379B00ECF9121E70901750E0FAA3E0D283F5A05B
:1037AB00C280D280EAF5A0C280D280C28390186911
:1037BB00E0F8A3E0F9901750E8F0A3E9F0850C824C
:1037CB00850D83E024F8F50AEEFAEFFBA90A121E29
:1037DB0070901750E0FAA3E0D283F5A0C280D2809C
:1037EB00EAF5A0C280D280C283850882850983E571
:1037FB000AF0EE24010EEF3400FF850C82850D8359
:10380B00A385820C85830D850882850983A3858218
:10381B0008858309850E82850F83A385820E858398
:10382B000FC3EE948FEF940150030237030221E292
:10383B0074F11202D8D2A8C290901743E0A2E450C0
:10384B00F8E0C2E4F0C2A8123366901000E0640204
:10385B0070087401901752F08009901752E07003B2
:10386B000239BD7E007F00750E79750F15750891B5
:10387B00750911E02415F50CE43415F50D75A6004A
:10388B0075A0FFC295E5A0245CF582E43404F583B2
:10389B00E493850E82850F83F0D29575A6FF85087C
:1038AB0082850983E0FC74786C600874C86E7001C3
:1038BB00EF700B90175074EFF0A3747B8052EC7584
:1038CB00F00584E5F07011EEF8EFF97A197B001230
:1038DB000207EA7001EB60DB8C0A7405250AF8E439
:1038EB003400F97A197B001201FFEA7001EB7011B9
:1038FB00EEF8EFF97A057B00120207EA7001EB6034
:10390B00B290174EE0F8A3E0F9901750E8F0A3E956
:10391B00F0EEFAEFFBECF9121E70901750E0FAA3E1
:10392B00E0D283F5A0C280D280EAF5A0C280D2801B
:10393B00C28390186BE0F8A3E0F9901750E8F0A35E
:10394B00E9F0850C82850D83E024F8F50AEEFAEF99
:10395B00FBA90A121E70901750E0FAA3E0D283F570
:10396B00A0C280D280EAF5A0C280D280C283850833
:10397B0082850983E50AF0EE24010EEF3400FF8502
:10398B000C82850D83A385820C85830D850882852A
:10399B000983A3858208858309850E82850F83A3FE
:1039AB0085820E85830FC3EE948FEF940150030233
:1039BB0038880221E274F11202D874FA120283D20F
:1039CB00A8C290901743E0A2E450F8E0C2E4F0C222
:1039DB00A812342F901000E0640270087401901745
:1039EB0052F08009901752E07003023CCF7E007FAB
:1039FB000074041202CE7485F0A37413F0740212D7
:103A0B0002CE7479F0A37415F0750C01750D107559
:103A1B000891750911901752E0F82421FAE4341338
:103A2B00FB851082851183EAF0A3EBF0E82415F5F2
:103A3B000EE43415F50F75A60075A0FFC297E5A02F
:103A4B00245CF582E43405F583E493C0E07404123E
:103A5B0002CEE0F8A3E0F5838882D0E0F0D297C2E3
:103A6B0095E5A0245CF582E43405F583E493C0E08E
:103A7B0074021202CEE0F8A3E0F5838882D0E0F066
:103A8B00D29575A6FF850C82850D83E0FC74786C4E
:103A9B00600874C86E7001EF700B90175074EFF0E4
:103AAB00A3747B8052EC75F00584E5F07011EEF891
:103ABB00EFF97A197B00120207EA7001EB60DB8CDD
:103ACB000A7405250AF8E43400F97A197B0012010F
:103ADB00FFEA7001EB7011EEF8EFF97A057B00123B
:103AEB000207EA7001EB60B290174EE0F8A3E0F921
:103AFB00901750E8F0A3E9F0EEFAEFFBECF9121E89
:103B0B0070901750E0FAA3E0D283F5A0C280D28068
:103B1B00EAF5A0C280D280C283850882850983E042
:103B2B00FC74786C600874C86E7001EF700B9017A2
:103B3B005074EFF0A3747B8052EC75F00584E5F0C4
:103B4B007011EEF8EFF97A197B00120207EA700197
:103B5B00EB60DB8C0A7405250AF8E43400F97A195A
:103B6B007B001201FFEA7001EB7011EEF8EFF97AAE
:103B7B00057B00120207EA7001EB60B290174EE072
:103B8B00F8A3E0F9901750E8F0A3E9F0EEFAEFFB99
:103B9B00ECF9121E70901750E0FAA3E0D283F5A057
:103BAB00C280D280EAF5A0C280D280C2839018690D
:103BBB00E0F8A3E0F9901750E8F0A3E9F085108244
:103BCB00851183E0F8A3E0F5838882E0246AF50A87
:103BDB00EEFAEFFBA90A121E70901750E0FAA3E061
:103BEB00D283F5A0C280D280EAF5A0C280D280C277
:103BFB0083850C82850D83E50AF090186BE0F8A3A2
:103C0B00E0F9901750E8F0A3E9F0850E82850F8359
:103C1B00E02406F50AEEFAEFFBA90A121E709017C4
:103C2B0050E0FAA3E0D283F5A0C280D280EAF5A0DF
:103C3B00C280D280C283850882850983E50AF0EEB3
:103C4B0024010EEF3400FF850E82850F83A385823E
:103C5B000E85830F851082851183E02401F8A3E084
:103C6B003400F9851082851183E8F0A3E9F085080B
:103C7B0082850983A3858208858309850C82850D3E
:103C8B0083A385820C85830D74021202CEE024017E
:103C9B00F8A3E03400F974021202CEE8F0A3E9F0C5
:103CAB0074041202CEE02401F8A3E03400F974048A
:103CBB001202CEE8F0A3E9F0C3EE948FEF9401501B
:103CCB0003023A41C296D29674061202990221E679
:103CDB0074F31202D8D2A8C290901743E0A2E4501A
:103CEB00F8E0C2E4F0C2A81235AD901000E0640217
:103CFB0070087401901752F08009901752E070030E
:103D0B00023E7D75A60075A0FF7E007F0078857949
:103D1B0013C297E5A0245CF582E43404F583E493A5
:103D2B0088828983F0D297C295E5A0245CF582E462
:103D3B003404F583E49388828983A3F0D295EE242F
:103D4B00020E0EEF3400FFE824020808E93400F9F4
:103D5B00C3EE948EEF940140B875A6FF7E007F00F2
:103D6B00750801750910901752E02421F50CE43405
:103D7B0013F50D850882850983E0FC74786C600867
:103D8B0074C86E7001EF700B90175074EFF0A37442
:103D9B007B8052EC75F00584E5F07011EEF8EFF9CD
:103DAB007A197B00120207EA7001EB60DB8C0A7454
:103DBB0005250AF8E43400F97A197B001201FFEAB1
:103DCB007001EB7011EEF8EFF97A057B0012020728
:103DDB00EA7001EB60B290174EE0F8A3E0F9901790
:103DEB0050E8F0A3E9F0EEFAEFFBECF9121E70903D
:103DFB001750E0FAA3E0D283F5A0C280D280EAF597
:103E0B00A0C280D280C28390175074FFF0A3F085BC
:103E1B000C82850D83E024F8F50AEEFAEFFBA90A74
:103E2B00121E70901750E0FAA3E0D283F5A0C28067
:103E3B00D280EAF5A0C280D280C283850882850930
:103E4B0083E50AF0EE24010EEF3400FF850C82852A
:103E5B000D83A385820C85830D850882850983A339
:103E6B00858208858309C3EE948FEF94015003027A
:103E7B003D7EC296D2967F0602033874F41202D8A6
:103E8B00901750E0F50AA3E0F50B901750E4F0A360
:103E9B0074F8F0901747E0A2E7E492E044FEF4FADE
:103EAB0090173EE02AF0901747E0A2E6E492E04438
:103EBB00FEF4FA90173EE0C39AF064FF70047408A6
:103ECB008007E0C394094002E4F0901759E0FA90A0
:103EDB00173EE06A60031224EB90186DE0F8A3E044
:103EEB00F990174EE8F0A3E9F090174C74FFF0A38C
:103EFB00F090173EE012038100088D45193F1F3FDC
:103F0B00963F1740A3402D41A7418F440D451245C5
:103F1B00A902458D901745E0C2E0F07E127F007537
:103F2B0008077C0D7D00EEFAEFFB79021223787CFB
:103F3B000D7D0074012EFAE43FFB7902122378EE1B
:103F4B00240AFEEF3400FF1508E50870D57E007FCC
:103F5B00007508148E09EE2404F582EF3418F583EE
:103F6B00E0FAEE24010EEF3400FFEAFC743F6A70B6
:103F7B0003024485AA08AB09790212207FE50824C5
:103F8B000AF508E5093400F50980CB901745E0C226
:103F9B00E0F07E587F0075080A7C0D7D00EEFAEF8D
:103FAB00FB79021223787C0D7D0074012EFAE43F1D
:103FBB00FB7902122378EE240AFEEF3400FF15087A
:103FCB00E50870D57E007F0075085A8E098015AA0A
:103FDB0008AB09790212207FE508240AF508E509E8
:103FEB003400F509EE240EF582EF3418F583E0FA70
:103FFB00EE24010EEF3400FFEAFC743F6A70D090A0
:10400B00174EE4F0A3F012469702458D901745E04A
:10401B00C2E0F07EBC7F0075080A7C0D7D00EEFAD5
:10402B00EFFB79021223787C0D7D0074012EFAE4EC
:10403B003FFB7902122378EE240AFEEF3400FF15C2
:10404B0008E50870D5901869E0F8A3E0F990174CD3
:10405B00E8F0A3E9F07E007F007508BE8E0980159D
:10406B00AA08AB09790212207FE508240AF508E5B6
:10407B00093400F509EE2418F582EF3418F583E0C6
:10408B00FAEE24010EEF3400FFEAFC743F6A70D0A5
:10409B007900124A4B02458D901745E0C2E0F07E45
:1040AB00207F0175080A7C0D7D00EEFAEFFB79028B
:1040BB001223787C0D7D0074012EFAE43FFB79020C
:1040CB00122378EE240AFEEF3400FF1508E5087082
:1040DB00D590186BE0F8A3E0F990174CE8F0A3E942
:1040EB00F07E007F007508227509018015AA08ABC8
:1040FB0009790212207FE508240AF508E509340046
:10410B00F509EE2422F582EF3418F583E0FAEE245C
:10411B00010EEF3400FFEAFC743F6A70D0790102A4
:10412B00409D901745E0C2E0F07E127F00750807B6
:10413B007C0D7D00EEFAEFFB79E11223787C0D7D8F
:10414B000074012EFAE43FFB79E1122378EE240A86
:10415B00FEEF3400FF1508E50870D57E007F007573
:10416B0008148E098015AA08AB0979E112207FE5A6
:10417B0008240AF508E5093400F509EE242CF5822C
:10418B00EF3418F583E0FAEE24010EEF3400FFEA6A
:10419B00FC743F6A70D012490602458D901745E0BA
:1041AB00C2E0F07E587F007508067C0D7D00EEFAAC
:1041BB00EFFB79E11223787C0D7D0074012EFAE47C
:1041CB003FFB79E1122378EE240AFEEF3400FF1552
:1041DB0008E50870D57E007F0075085A8E0980159A
:1041EB00AA08AB0979E112207FE508240AF508E556
:1041FB00093400F509EE2436F582EF3418F583E027
:10420B00FAEE24010EEF3400FFEAFC743F6A70D023
:10421B00901743E0A2E74003024304901747E0A244
:10422B00E550030243E7901743E0C2E7F090174EC7
:10423B00E4F0A3F075088F75090178081203707C00
:10424B00DE7A007B007914121F937402120299120A
:10425B00240E7E537F17901741E0F8A3E0F9E87521
:10426B00F006A4F8AAF075F006E9A42AF9E8247C74
:10427B00FAE93418FBEAF8EBF97C047D18750805AC
:10428B0088828983E493F5098E828F83F0EC240B6B
:10429B00F582ED3400F583E509F08C828D83A3ACB8
:1042AB0082AD8388828983A3A882A9838E828F8320
:1042BB00A3AE82AF831508E50870C58A828B83A3F2
:1042CB00A3A3A3A3E493901758F090174EE4F0A385
:1042DB00F07582537583177E64FFE0FAFC743F6AB6
:1042EB0070030243E7EEFAEFFB790212207FEE2414
:1042FB000AFEEF3400FFA380E1E0A2E75003024384
:10430B00E7901747E0A2E450030243E7901743E01E
:10431B00D2E7F090174EE4F0A3F075088F75090102
:10432B0078081203707CDE7A007B007914121F93DD
:10433B00740212029912240E7E537F17901741E0DC
:10434B00F8A3E0F9E875F006A4F8AAF075F006E911
:10435B00A42AF9E82424FAE93419FBEAF8EBF97CEE
:10436B00047D1875080588828983E493F5098E828C
:10437B008F83F0EC240BF582ED3400F583E509F027
:10438B008C828D83A3AC82AD8388828983A3A88220
:10439B00A9838E828F83A3AE82AF831508E5087045
:1043AB00C58A828B83A3A3A3A3A3E493901758F08E
:1043BB0090174EE4F0A3F07582537583177E64FF5C
:1043CB008012EEFAEFFB790212207FEE240AFEEF49
:1043DB003400FFA3E0FAFC743F6A70E690174EE4DA
:1043EB00F0A374F8F0901743E0A2E75038C2B07412
:1043FB0080901870F090174C74E0F0A37407F07570
:10440B0082EE7583177E647F00E0FAFC743F6A606E
:10441B0069EEFAEFFB79E112207FEE240AFEEF340E
:10442B0000FFA380E4901744E0FAE0FBEAA2E0501F
:10443B0009EBA2E150047440800CE0A2E04005E0DF
:10444B00A2E150067480901870F0D2B090174C74A3
:10445B00FFF0A3F07582EE7583177E647F008012E8
:10446B00EEFAEFFB79E112207FEE240AFEEF340027
:10447B00FFA3E0FAFC743F6A70E690174EE4F0A3DA
:10448B00F002458D901745E0C2E0F07E947F0075F9
:10449B0008087C0D7D00EEFAEFFB79E11223787CA6
:1044AB000D7D0074012EFAE43FFB79E1122378EEC7
:1044BB00240AFEEF3400FF1508E50870D57E007F57
:1044CB00007508968E098015AA08AB0979E11220B0
:1044DB007FE508240AF508E5093400F509EE2440C8
:1044EB00F582EF3418F583E0FAEE24010EEF340079
:1044FB00FFEAFC743F6A70D090174EE4F0A3F0F91A
:10450B00807D901745E0C2E0F07EE47F00750808DF
:10451B007C0D7D00EEFAEFFB79E11223787C0D7DAB
:10452B000074012EFAE43FFB79E1122378EE240AA2
:10453B00FEEF3400FF1508E50870D57E007F00758F
:10454B0008E68E098015AA08AB0979E112207FE5F0
:10455B0008240AF508E5093400F509EE244AF5822A
:10456B00EF3418F583E0FAEE24010EEF3400FFEA86
:10457B00FC743F6A70D090174EE4F0A3F0790112EF
:10458B0049C790174EE4F0A3F0901750E50AF0A33B
:10459B00E50BF090173EE0901759F002342A74F7B0
:1045AB001202D8901743E0A2E750030246949017EB
:1045BB0047E0A2E05005E0A2E1402590174EE4F061
:1045CB00A3F075088F75090178081203707CDE7AE9
:1045DB00007B007914121F93740212029912240E9D
:1045EB00901744E0FAE0FBEAA2E05025EBA2E15081
:1045FB0020901747E0A2E04007901744E0C2E0F09C
:10460B00901747E0A2E1405C901744E0C2E1F080D4
:10461B0053E0A2E0501F901747E0A2E0400790172D
:10462B0044E0C2E0F0901747E0A2E1403790174416
:10463B00E0D2E180D9E0A2E1901747E05015A2E06B
:10464B004007901744E0D2E0F0901747E0A2E1401A
:10465B001380B5A2E04008901744E0D2E080AFE0B1
:10466B00A2E150C9901744E0FAE0FBEAA2E050093E
:10467B00EBA2E150047440800CE0A2E04005E0A204
:10468B00E150067480901870F002490174F7120221
:10469B00D890174C74FFF0A3F0901747E0A2E450AA
:1046AB0003024738901748E0A2E09017415025E0ED
:1046BB002401F0A3E03400F0901741C3E0941CA355
:1046CB00E09400A2D265D033403C901741741BF0AC
:1046DB00A3E48031C3E09418A3E09400A2D265D088
:1046EB0033901741E040102401F0A3E03400F09028
:1046FB001748E0D2E0800E2401F0A3E03400F090E4
:10470B001748E0C2E0F0901748E0C2E1F0E0A2E108
:10471B005054741890173FF07440901740F0740287
:10472B00901736F0901748E0D2E2024813E0A2E56A
:10473B00402B901741E024FFF0F8A3E034FFF0F991
:10474B00C3E89401E99400A2D265D03350B8901716
:10475B0041E4F0A3F0901748E0D2E180AF90174E00
:10476B00E4F0A3024900E0A2E0504C901741E0F5C1
:10477B0008A3E0F50978081203B7180003BE4792A7
:10478B0047A547A947B247741890173FF0E4901715
:10479B0040F0901748E0C2E080187418800B741931
:1047AB0090173FF0E48008741990173FF0748090D5
:1047BB001740F07402804EE0A2E25004741880E0BF
:1047CB00901741E0F8A3E0F9E8C333F8E933F9E8CF
:1047DB002444F582E93418F583E493C0E074019323
:1047EB00F583D082AA82AB838A088B09740278087E
:1047FB00120260E50890173FF0EAC4333354C090BF
:10480B001740F07401901736F07508007E537F1730
:10481B00901741E0F8A3E0F9E875F006A4F8AAF0C8
:10482B0075F006E9A42AF9E82424FAE93419FBE81F
:10483B00247CF8E93418F97C047D18901743E0A226
:10484B00E750068A828B83800488828983E4938E67
:10485B00828F83F0E508C394055010E0C0E0EC2490
:10486B000BF582ED3400F583D0E0F005088C828DDA
:10487B0083A3AC82AD8388828983A3A882A9838A10
:10488B00828B83A3AA82AB838E828F83A3AE82AFEC
:10489B0083E508C3940640A390174EE4F0A374F885
:1048AB00F07582537583177E647F008012EEFAEFEA
:1048BB00FB790212207FEE240AFEEF3400FFA3E007
:1048CB00FAFC743F6A70E690174EE4F0A3F0901771
:1048DB003FE0901737F0901740E0901738F09017A3
:1048EB0043E0C2E3F0E0D2E2F0901746E0D2E1F011
:1048FB007459901802F07F0202033874F81202D830
:10490B00901747E0A2E0404D901000E06016901821
:10491B0069E0F8A3E0F990174CE8F0A3E9F0E49014
:10492B001000800A7402F090174C74FFF0A3F0751E
:10493B0082F37583177E1E7F00E0FAFC743F6A607A
:10494B0069EEFAEFFB79E112207FEE240AFEEF34D9
:10495B0000FFA380E4E0A2E14050901000E064016E
:10496B00601790186BE0F8A3E0F990174CE8F0A3F0
:10497B00E9F07401901000800A7402F090174C74E7
:10498B00FFF0A3F07582F37583177E1E7F008012F4
:10499B00EEFAEFFB79E112207FEE240AFEEF3400F2
:1049AB00FFA3E0FAFC743F6A70E690174EE4F0A3A5
:1049BB00F090174C74FFF0A3F002237374F71202FC
:1049CB00D8901747E0A2E04055E9705290174EE49B
:1049DB00F0A3F075088F75090178081203707CDE5F
:1049EB007A007B007914121F9374021202999017AC
:1049FB004C74FFF0A3F07582F97583177E147F005A
:104A0B008012EEFAEFFB79BE12207FEE240AFEEF46
:104A1B003400FFA3E0FAFC743F6A70E680FEE0A26C
:104A2B00E440047A018007E0A2E540117AFFE970C7
:104A3B0007EA25EAF5EA8005EA25FCF5FC024901BF
:104A4B0074F71202D8E96003024B60901747E0A29B
:104A5B00E4400F901871E004F0C3940840197407F8
:104A6B008014E0A2E55003024C81901871E014F021
:104A7B00C394C94002E4F07E007A537B1778047923
:104A8B00188E08901871E075F005A4241CFCE5F055
:104A9B003418FDE5082CF582E43DF583E4938A8216
:104AAB008B83F0C0E0E82415F582E93400F583D060
:104ABB00E0F00E88828983A3A882A9838A828B83E4
:104ACB00A3AA82AB83EEC3940440B6901871E07531
:104ADB00F005A42420F582E5F03418F583E49390D7
:104AEB001757F07582537583177EC87F008012EEBF
:104AFB00FAEFFB790212207FEE240AFEEF3400FF5F
:104B0B00A3E0FAFC743F6A70E6901871E0FEC39460
:104B1B000590173AE04004C2E08002D2E0F0901713
:104B2B0046E054EDF090173AE0901736F0795D12AD
:104B3B0028C2901746E054EDF0EEC333F8E433F996
:104B4B00E8240CF582E93418F583E493901736F0DA
:104B5B007948024C6F7401696003024C72901747DD
:104B6B00E0A2E4400F901872E004F0C394084019DF
:104B7B0074078014E0A2E55003024C81901872E098
:104B8B0014F0C394C94002E4F07E007A537B17788B
:104B9B000479188E08901872E075F005A4241CFC9B
:104BAB00E5F03418FDE5082CF582E43DF583E4933C
:104BBB008A828B83F0C0E0E8241FF582E93400F58C
:104BCB0083D0E0F00E88828983A3A882A9838A828E
:104BDB008B83A3AA82AB83EEC3940440B690187266
:104BEB00E075F005A42420F582E5F03418F583E494
:104BFB0093901757F07582537583177E2C7F018026
:104C0B0012EEFAEFFB790212207FEE240AFEEF344C
:104C1B0000FFA3E0FAFC743F6A70E6901872E0FEA6
:104C2B00C3940590173AE04004C2E18002D2E1F050
:104C3B00901746E054EDF090173AE0901736F07964
:104C4B005D1228C2901746E054EDF0EEC333F8E442
:104C5B0033F9E8240CF582E93418F583E4939017C3
:104C6B0036F079491228C290174EE4F0A3F0901752
:094C7B004C74FFF0A3F0024901A2
:040000050000009166
:00000001FF
